:020000040000FA
:0408000063EF09F0A9
:1008100003B283EF05F0F2B4A1EF05F09EB0A9EFAB
:1008200005F09EB2B1EF05F0F2A81AEF04F0F2B2B3
:1008300032EF04F09EB61FEF04F012EF09F09E961F
:1008400000011450000A06E000011450010A06E0FD
:1008500012EF09F07DEC20F012EF09F075EC22F0B8
:1008600012EF09F0CD90F2929EA03CEF04F001014E
:10087000533F3CEF04F0542BAEC1B2F1AFC1B3F122
:10088000B0C1B4F1B1C1B5F1AAC1AEF1ABC1AFF124
:10089000ACC1B0F1ADC1B1F1A6C1AAF1A7C1ABF134
:1008A000A8C1ACF1A9C1ADF1A2C1A6F1A3C1A7F144
:1008B000A4C1A8F1A5C1A9F19EC1A2F19FC1A3F154
:1008C000A0C1A4F1A1C1A5F19AC19EF19BC19FF164
:1008D0009CC1A0F19DC1A1F196C19AF197C19BF174
:1008E00098C19CF199C19DF1CECF96F1CFCF97F1F0
:1008F00053C198F154C199F1CF6ACE6A0101536B8B
:10090000546B9E90CD800FBC0F8E0FBA8BEF04F00E
:100910000F8A12EF09F00F8C0FBEC7EF04F096C1DB
:100920009AF197C19BF198C19CF199C19DF19AC12F
:100930009EF19BC19FF19CC1A0F19DC1A1F19EC1FF
:10094000A2F19FC1A3F1A0C1A4F1A1C1A5F1A2C1CF
:10095000A6F1A3C1A7F1A4C1A8F1A5C1A9F1A6C19F
:10096000AAF1A7C1ABF1A8C1ACF1A9C1ADF1AAC16F
:10097000AEF1ABC1AFF1ACC1B0F1ADC1B1F1AEC13F
:10098000B2F1AFC1B3F1B0C1B4F1B1C1B5F1010180
:100990005E6B5F6B606B616B96515E2797515F2357
:1009A00098516023995161239A515E279B515F238F
:1009B0009C5160239D5161239E515E279F515F236F
:1009C000A0516023A1516123A2515E27A3515F234F
:1009D000A4516023A5516123A6515E27A7515F232F
:1009E000A8516023A9516123AA515E27AB515F230F
:1009F000AC516023AD516123AE515E27AF515F23EF
:100A0000B0516023B1516123B2515E27B3515F23CE
:100A1000B4516023B5516123D89001016133603333
:100A20005F335E33D8900101613360335F335E33EF
:100A3000D8900101613360335F335E3300C10CF144
:100A400001C10DF102C10EF103C10FF104C110F19A
:100A500005C111F106C112F107C113F108C114F16A
:100A600009C115F10AC116F10BC117F134C135F1F5
:100A700011B846EF05F00101620E046F010E056F1B
:100A8000000E066F000E076F4FEF05F00101A70E75
:100A9000046F020E056F000E066F000E076F5EC139
:100AA00000F15FC101F160C102F161C103F114EC19
:100AB0001FF003BF04D019BE02D019A0108C11A0E2
:100AC00067EF05F010BA67EF05F00F80108A0CC1D0
:100AD00000F10DC101F10EC102F10FC103F110C10E
:100AE00004F111C105F112C106F113C107F114C1DE
:100AF00008F115C109F116C10AF117C10BF135C191
:100B000034F112EF09F00392ABB2AB98AB8803015A
:100B100003EE00F080517F0BE92604C0EFFF802B2D
:100B20008151805D700BD8A48B8200008051815D63
:100B3000700BD8A48B9281518019D8B4079012EF12
:100B400009F0F2940101453F12EF09F0462B12EF34
:100B500009F09E900101533F12EF09F0542B12EF60
:100B600009F09E9211B820EF07F08BB4BFEF05F0AB
:100B700010ACBFEF05F08B84109CC0EF05F08B9498
:100B8000C3CF55F1C4CF56F1C28207B42AEF06F0A5
:100B900047C14BF148C14CF149C14DF14AC14EF139
:100BA0005EC162F15FC163F160C164F161C165F171
:100BB00096C1B6F197C1B7F198C1B8F199C1B9F131
:100BC0009AC1BAF19BC1BBF19CC1BCF19DC1BDF101
:100BD0009EC1BEF19FC1BFF1A0C1C0F1A1C1C1F1D1
:100BE000A2C1C2F1A3C1C3F1A4C1C4F1A5C1C5F1A1
:100BF000A6C1C6F1A7C1C7F1A8C1C8F1A9C1C9F171
:100C0000AAC1CAF1ABC1CBF1ACC1CCF1ADC1CDF140
:100C1000AEC1CEF1AFC1CFF1B0C1D0F1B1C1D1F110
:100C2000B2C1D2F1B3C1D3F1B4C1D4F1B5C1D5F1E0
:100C3000010155515B2756515C23E86A5D230E2E56
:100C40002AEF06F05CC157F15DC158F15B6B5C6B3C
:100C50005D6B078E0201002F12EF09F03C0E006F52
:100C60001A50E00BE00AE866128818BE02D018B4E9
:100C7000108E00C10CF101C10DF102C10EF103C1D2
:100C80000FF104C110F105C111F106C112F107C144
:100C900013F108C114F109C115F10AC116F10BC114
:100CA00017F134C135F101018A675EEF06F08B67F9
:100CB0005EEF06F08C675EEF06F08D6762EF06F080
:100CC00092EF06F08EC100F18FC101F190C102F1E7
:100CD00091C103F10101010E046F000E056F000EBA
:100CE000066F000E076F14EC1FF000C18EF101C1FA
:100CF0008FF102C190F103C191F1006787EF06F017
:100D0000016787EF06F0026787EF06F0036792EF4F
:100D100006F08AC18EF18BC18FF18CC190F18DC12B
:100D200091F10F80D57ED5BE6DD0D6CF47F1D7CF0C
:100D300048F145C149F1E86AE8CF4AF119BE02D04D
:100D400019A0108C109047C100F148C101F149C1B0
:100D500002F14AC103F101010A0E046F000E056F92
:100D6000000E066F000E076F14EC1FF003AF10802B
:100D7000010154A7C8EF06F00F9A0F9C0F9E0101C6
:100D8000000E5E6F600E5F6F3D0E606F080E616F4C
:100D9000010147BFD8EF06F04867D8EF06F0496772
:100DA000D8EF06F04A67D8EF06F0F288FDEF06F0BC
:100DB000F2985E6B5F6B606B616B966B976B986B79
:100DC000996B9A6B9B6B9C6B9D6B9E6B9F6BA06BE7
:100DD000A16BA26BA36BA46BA56BA66BA76BA86B97
:100DE000A96BAA6BAB6BAC6BAD6BAE6BAF6BB06B47
:100DF000B16BB26BB36BB46BB56BD76AD66A0101DA
:100E0000456B466B0CC100F10DC101F10EC102F141
:100E10000FC103F110C104F111C105F112C106F1B6
:100E200013C107F114C108F115C109F116C10AF186
:100E300017C10BF135C134F112EF09F012EF09F0CF
:100E40000201002F79EF08F0D59ED6CF47F1D7CF1A
:100E500048F145C149F1E86AE8CF4AF1D76AD66A54
:100E60000101456B466BD58E1A50E00BE00AE8662F
:100E7000128818BE02D018B4108E17AE1C8C00C198
:100E80000CF101C10DF102C10EF103C10FF104C15A
:100E900010F105C111F106C112F107C113F108C12A
:100EA00014F109C115F10AC116F10BC117F134C1D2
:100EB00035F10FA0109A11B869EF07F00101620E29
:100EC000046F010E056F000E066F000E076F72EFC4
:100ED00007F00101A70E046F020E056F000E066FEA
:100EE000000E076F47C100F148C101F149C102F18D
:100EF0004AC103F114EC1FF003BF85EF07F019BEE0
:100F000002D019A0108C11B00F800CC100F10DC1DE
:100F100001F10EC102F10FC103F110C104F111C1C1
:100F200005F112C106F113C107F114C108F115C191
:100F300009F116C10AF117C10BF135C134F10201F3
:100F40003C0E006F00C10CF101C10DF102C10EF1A8
:100F500003C10FF104C110F105C111F106C112F175
:100F600007C113F108C114F109C115F10AC116F145
:100F70000BC117F134C135F101018A67C7EF07F0E2
:100F80008B67C7EF07F08C67C7EF07F08D67CBEF74
:100F900007F0FBEF07F08EC100F18FC101F190C1A6
:100FA00002F191C103F10101010E046F000E056F02
:100FB000000E066F000E076F14EC1FF000C18EF1DB
:100FC00001C18FF102C190F103C191F10067F0EF0F
:100FD00007F00167F0EF07F00267F0EF07F0036733
:100FE000FBEF07F08AC18EF18BC18FF18CC190F1BC
:100FF0008DC191F10F80109047C100F148C101F1FE
:1010000049C102F14AC103F101010A0E046F000E49
:10101000056F000E066F000E076F14EC1FF003AF94
:101020001080010154A721EF08F00F9A0F9C0F9E2A
:101030000101000E5E6F600E5F6F3D0E606F080E67
:10104000616F47C100F148C101F149C102F14AC1D4
:1010500003F10101140E046F050E056F000E066FFB
:10106000000E076F14EC1FF003AF3AEF08F0F288A0
:101070005FEF08F0F2985E6B5F6B606B616B966B75
:10108000976B986B996B9A6B9B6B9C6B9D6B9E6B34
:101090009F6BA06BA16BA26BA36BA46BA56BA66BE4
:1010A000A76BA86BA96BAA6BAB6BAC6BAD6BAE6B94
:1010B000AF6BB06BB16BB26BB36BB46BB56B0CC198
:1010C00000F10DC101F10EC102F10FC103F110C118
:1010D00004F111C105F112C106F113C107F114C1E8
:1010E00008F115C109F116C10AF117C10BF135C19B
:1010F00034F134EC23F01D661ED01CAE11D01C9EC2
:101100001D8E18AE07D0146A040E156E166A7DEC9B
:1011100020F011D0146A156A166A7DEC20F00BD00D
:101120001CAC09D01C9C1D8C010E146E156A166A2D
:1011300075EC22F000D08BB4A5EF08F010ACA5EF51
:1011400008F08B84109CA6EF08F08B94C3CF55F168
:10115000C4CF56F1C28207B410EF09F047C14BF17A
:1011600048C14CF149C14DF14AC14EF15EC162F135
:101170005FC163F160C164F161C165F196C1B6F10F
:1011800097C1B7F198C1B8F199C1B9F19AC1BAF153
:101190009BC1BBF19CC1BCF19DC1BDF19EC1BEF123
:1011A0009FC1BFF1A0C1C0F1A1C1C1F1A2C1C2F1F3
:1011B000A3C1C3F1A4C1C4F1A5C1C5F1A6C1C6F1C3
:1011C000A7C1C7F1A8C1C8F1A9C1C9F1AAC1CAF193
:1011D000ABC1CBF1ACC1CCF1ADC1CDF1AEC1CEF163
:1011E000AFC1CFF1B0C1D0F1B1C1D1F1B2C1D2F133
:1011F000B3C1D3F1B4C1D4F1B5C1D5F10101555199
:101200005B2756515C23E86A5D230E2E10EF09F030
:101210005CC157F15DC158F15B6B5C6B5D6B078E18
:1012200012EF09F002C0E0FF005001C0D8FF10002B
:10123000A6B218EF09F00CC0A9FF0BC0A8FFA69E2C
:10124000A69CA684F29E550EA76EAA0EA76EA68235
:10125000F28EA694A6B22AEF09F00C2A1200A96E0B
:10126000A69EA69CA680A8500C2A120004012C0E53
:10127000826F3BEC0BF00FEC20F00C502FEC09F0E0
:10128000E8CF00F10C502FEC09F0E8CF01F101AFED
:101290004FEF09F00101FF0E026FFF0E036FB2EC7A
:1012A0001FF029675BEF09F00401200E826F3BEC11
:1012B0000BF060EF09F004012D0E826F3BEC0BF098
:1012C000BCEC1DF01200306A076A0F6A106A116ADE
:1012D000126A136A0F010E0EC16E860EC06E030EE7
:1012E000C26E0F01896A110E926E080E8A6EF10E9F
:1012F000936E8B6A980E946EF18EFC0E2FEC09F0B3
:10130000E8CF0BF00BA011800BA211820BA411846B
:101310000BA81188C90E2FEC09F0E8CF17F0CA0E00
:101320002FEC09F0E8CF18F0CB0E2FEC09F0E8CF46
:1013300019F0CC0E2FEC09F0E8CF1AF0CD0E2FECFF
:1013400009F0E8CF2FF01C6A1D6A0E6A01015B6B81
:101350005C6B5D6B576B586BF29A0101476B486B86
:10136000496B4A6B4B6B4C6B4D6B4E6B4F6B506BC1
:10137000516B526B456B466BD76AD66A0F01280ECC
:10138000D56EF28A9D90B00ECD6E01015E6B5F6BE3
:10139000606B616B626B636B646B656B666B676BD9
:1013A000686B696B536B546BCF6ACE6A0F9A0F9C54
:1013B0000F9E9D80760ECA6E9D8202013C0E006FCC
:1013C000CC6A160E2FEC09F0E8CF00F1170E2FECC7
:1013D00009F0E8CF01F1180E2FEC09F0E8CF02F187
:1013E000190E2FEC09F0E8CF03F1010103AF13EF61
:1013F0000AF00FEC20F0160E0C6E00C10BF018EC8A
:1014000009F0170E0C6E01C10BF018EC09F0180E64
:101410000C6E02C10BF018EC09F0190E0C6E03C132
:101420000BF018EC09F000C18AF101C18BF102C187
:101430008CF103C18DF100C18EF101C18FF102C1A8
:1014400090F103C191F11A0E2FEC09F0E8CF00F1F1
:101450001B0E2FEC09F0E8CF01F11C0E2FEC09F068
:10146000E8CF02F11D0E2FEC09F0E8CF03F10101E6
:1014700003AF69EF0AF00FEC20F01A0E0C6E00C1FA
:101480000BF018EC09F01B0E0C6E01C10BF018EC00
:1014900009F01C0E0C6E02C10BF018EC09F01D0EC9
:1014A0000C6E03C10BF018EC09F01A0E2FEC09F0CA
:1014B000E8CF00F11B0E2FEC09F0E8CF01F11C0E74
:1014C0002FEC09F0E8CF02F11D0E2FEC09F0E8CF68
:1014D00003F100C192F101C193F102C194F103C182
:1014E00095F1240EAC6E900EAB6E240EAC6E080E11
:1014F000B86E000EB06E1F0EAF6E0401806B816B74
:101500000F01900EAB6E0F019D8A0301806B816B02
:10151000C26B8B92146A156A166A9D860790000149
:10152000F28EF28C07B065EF1CF00FB0FDEF15F0F6
:1015300010BEFDEF15F012B8FDEF15F0030180515C
:1015400081197F0BD8B465EF1CF013EE00F08151C8
:101550007F0BE126812BE7CFE8FFE00BD8B465EFE6
:101560001CF023EE82F0C2513F0BD926E7CFDFFFFC
:10157000C22BDF50780AD8A465EF1CF007808EC11B
:1015800000F18FC101F190C102F191C103F101019C
:10159000040E046F000E056F000E066F000E076F3D
:1015A00014EC1FF000AFDEEF0AF00101030E8E6FA6
:1015B000000E8F6F000E906F000E916F030182512D
:1015C000720AD8B4E1EF15F08251520AD8B4E1EFB3
:1015D00015F08251750AD8B4E1EF15F08251630A13
:1015E000D8B41FEF19F08251690AD8B488EF12F00D
:1015F00082517A0AD8B49BEF13F08251490AD8B4C9
:1016000027EF12F08251500AD8B431EF11F0825115
:10161000700AD8B479EF11F08251540AD8B4A9EF06
:1016200011F08251740AD8B4F4EF11F08251410ADA
:10163000D8B451EF0CF082514B0AD8B44FEF0BF0F5
:1016400082516D0AD8B484EF10F082514D0AD8B49B
:101650009DEF10F08251730AD8B411EF15F082514A
:10166000530AD8B476EF15F08251590AD8B4D5EFA1
:101670000FF056EF19F0040114EE00F080517F0BCB
:10168000E12682C4E7FF802B120004010D0E826F59
:101690003BEC0BF00A0E826F3BEC0BF012000401E6
:1016A0004B0E826F3BEC0BF004012C0E826F3BEC77
:1016B0000BF081B802D02FB630D003018351430A1A
:1016C000D8B494EF0BF003018351630AD8B496EFBA
:1016D0000BF003018351520AD8B498EF0BF00301C9
:1016E0008351720AD8B49AEF0BF003018351470A71
:1016F000D8B49CEF0BF003018351670AD8B49EEF76
:101700000BF003018351540AD8B4A0EF0BF003018E
:101710008351740AD8B40FEF0CF003018351550ABA
:10172000D8B4A2EF0BF082D02F807AD02F9078D04F
:101730002F8276D02F9274D02F8472D02F9470D0B5
:101740002F866ED084C330F185C331F186C332F168
:1017500087C333F10101296B5DEC20F0D4EC1FF05D
:1017600000C104F101C105F102C106F103C107F195
:1017700050EC20F0200EF86EF76AF66A0900F5CFFB
:101780002CF10900F5CF2DF10900F5CF2EF109005C
:10179000F5CF2FF10900F5CF30F10900F5CF31F188
:1017A0000900F5CF32F10900F5CF33F10101296BC2
:1017B0005DEC20F0D4EC1FF014EC1FF00067E8EFB4
:1017C0000BF00167E8EF0BF00267E8EF0BF003673F
:1017D00001D025D004014E0E826F3BEC0BF00401CA
:1017E0006F0E826F3BEC0BF004014D0E826F3BECF1
:1017F0000BF00401610E826F3BEC0BF00401740EE0
:10180000826F3BEC0BF00401630E826F3BEC0BF03C
:101810000401680E826F3BEC0BF054EF19F02F9629
:10182000CD0E0C6E2FC00BF018EC09F0CD0E2FEC86
:1018300009F0E8CF2FF02FB006D00401630E826FBD
:101840003BEC0BF005D00401430E826F3BEC0BF038
:101850002FB206D00401720E826F3BEC0BF005D064
:101860000401520E826F3BEC0BF02FB406D0040142
:10187000670E826F3BEC0BF005D00401470E826FC0
:101880003BEC0BF02FB606D00401740E826F3BECDC
:101890000BF005D00401540E826F3BEC0BF054EFBB
:1018A00019F00401410E826F3BEC0BF003018351F0
:1018B000310AD8B4F5EF0EF003018351320AD8B4DF
:1018C00025EF0EF003018351330AD8B4AEEF0DF0CB
:1018D00003018351340AD8B49EEF0CF00301835105
:1018E000350AD8B47BEF0CF004013F0E826F3BEC5D
:1018F0000BF054EF19F004012C0E826F3BEC0BF04F
:1019000003018451300AD8B48EEF0CF003018451E6
:10191000310AD8B496EF0CF0E7EF0DF08B9004018C
:10192000300E826F3BEC0BF09CEF0CF08B800401CF
:10193000310E826F3BEC0BF054EF19F0CC0E2FEC14
:1019400009F0E8CF0BF004012C0E826F3BEC0BF09A
:1019500003018451310AD8B4C2EF0CF00301845161
:10196000300AD8B4C4EF0CF0030184514D0AD8B446
:10197000CEEF0CF003018451540AD8B4D5EF0CF02B
:10198000ECEF0CF08A8401D08A940BAE04D00BAC3F
:1019900002D00BBA21D0E00E0B1218D01F0E0B167E
:1019A0008539E844E00B0B1211D0E00E0B1650EC19
:1019B00020F085C332F186C333F10101296B5DEC60
:1019C00020F0D4EC1FF000511F0B0B12CC0E0C6E4C
:1019D0000BC00BF018EC09F00401340E826F3BECE5
:1019E0000BF004012C0E826F3BEC0BF0CC0E2FECB5
:1019F00009F0E8CF1AF08AB406D00401300E826FE5
:101A00003BEC0BF005D00401310E826F3BEC0BF088
:101A100004012C0E826F3BEC0BF01A38E840070BE8
:101A2000E8CF82F40401300E82273BEC0BF0040176
:101A30002C0E826F3BEC0BF00FEC20F01A501F0BBA
:101A4000E8CF00F1B2EC1FF032C182F40401300E95
:101A500082273BEC0BF033C182F40401300E822765
:101A60003BEC0BF004012C0E826F3BEC0BF00FEC07
:101A700020F02DC000F100AF0BD0FF0E016FFF0E64
:101A8000026FFF0E036F04012D0E826F3BEC0BF013
:101A9000B2EC1FF031C182F40401300E82273BEC1E
:101AA0000BF032C182F40401300E82273BEC0BF0C4
:101AB00033C182F40401300E82273BEC0BF00401A9
:101AC0002C0E826F3BEC0BF00FEC20F02CC000F1E1
:101AD000B2EC1FF031C182F40401300E82273BECDE
:101AE0000BF032C182F40401300E82273BEC0BF084
:101AF00033C182F40401300E82273BEC0BF0040169
:101B00002C0E826F3BEC0BF00FEC20F02EC000F19E
:101B100000AF0BD0FF0E016FFF0E026FFF0E036FC1
:101B200004012D0E826F3BEC0BF0B2EC1FF031C1C3
:101B300082F40401300E82273BEC0BF032C182F4B8
:101B40000401300E82273BEC0BF033C182F4040118
:101B5000300E82273BEC0BF054EF19F0CB0E2FEC3C
:101B600009F0E8CF0BF004012C0E826F3BEC0BF078
:101B700003018451450AD8B4D2EF0DF0030184511A
:101B8000440AD8B4D5EF0DF003018451300AD8B41B
:101B9000D8EF0DF003018451310AD8B4DCEF0DF019
:101BA000E7EF0DF00B9EE1EF0DF00B8EE1EF0DF086
:101BB000FC0E0B16E1EF0DF0FC0E0B160B80E1EFA7
:101BC0000DF0CB0E0C6E0BC00BF018EC09F00401FD
:101BD000330E826F3BEC0BF004012C0E826F3BEC5A
:101BE0000BF0CB0E2FEC09F0E8CF19F019BE00EF87
:101BF0000EF00401450E826F3BEC0BF005EF0EF08A
:101C00000401440E826F3BEC0BF004012C0E826F3A
:101C10003BEC0BF00401300E826F3BEC0BF0040147
:101C20002C0E826F3BEC0BF019B01EEF0EF004018E
:101C3000300E826F3BEC0BF023EF0EF00401310EFF
:101C4000826F3BEC0BF054EF19F0CA0E2FEC09F049
:101C5000E8CF0BF004012C0E826F3BEC0BF003017C
:101C60008451450AD8B461EF0EF003018451440A4F
:101C7000D8B464EF0EF0030184514D0AD8B46DEF6F
:101C80000EF003018451410AD8B467EF0EF003014E
:101C90008451460AD8B46AEF0EF003018451560A03
:101CA000D8B475EF0EF003018451500AD8B480EF18
:101CB0000EF003018451520AD8B483EF0EF08CEF7A
:101CC0000EF00B9E86EF0EF00B8E86EF0EF00B9C47
:101CD00086EF0EF00B8C86EF0EF0FC0E0B1685C314
:101CE000E8FF030B0B1286EF0EF0C70E0B1685C331
:101CF000E8FF070BE846E846E8460B1286EF0EF0D1
:101D00000B8486EF0EF00B9486EF0EF0CA0E0C6E6D
:101D10000BC00BF018EC09F0CA0E2FEC09F0E8CF5D
:101D200018F00401320E826F3BEC0BF004012C0E14
:101D3000826F3BEC0BF018BEA5EF0EF00401450ED0
:101D4000826F3BEC0BF0AAEF0EF00401440E826FA1
:101D50003BEC0BF004012C0E826F3BEC0BF018C037
:101D6000E8FF030BE8CF82F40401300E82273BEC3E
:101D70000BF004012C0E826F3BEC0BF018BCC8EF8B
:101D80000EF00401410E826F3BEC0BF0CDEF0EF034
:101D90000401460E826F3BEC0BF004012C0E826FA7
:101DA0003BEC0BF018C0E8FF380BE842E842E84291
:101DB000E8CF82F40401300E82273BEC0BF00401E3
:101DC0002C0E826F3BEC0BF018B4EEEF0EF004011A
:101DD000520E826F3BEC0BF0F3EF0EF00401500E4D
:101DE000826F3BEC0BF054EF19F0C90E2FEC09F0A9
:101DF000E8CF0BF004012C0E826F3BEC0BF00301DB
:101E00008451450AD8B413EF0FF003018451440AFA
:101E1000D8B416EF0FF0030184514D0AD8B419EF6E
:101E20000FF027EF0FF00B9E21EF0FF00B8E21EF3D
:101E30000FF0F80E0B1685C3E8FF070B0B1221EF0E
:101E40000FF0C90E0C6E0BC00BF018EC09F004017A
:101E5000310E826F3BEC0BF004012C0E826F3BECD9
:101E60000BF0C90E2FEC09F0E8CF17F017BE06D023
:101E70000401450E826F3BEC0BF005D00401440ECB
:101E8000826F3BEC0BF004012C0E826F3BEC0BF0ED
:101E900017C0E8FF070BE8CF82F40401300E822759
:101EA0003BEC0BF004012C0E826F3BEC0BF0078037
:101EB0000FEC20F028C0E8FF003B00430043030B79
:101EC000B2EC1FF033C182F40401300E82273BECE8
:101ED0000BF004012C0E826F3BEC0BF00FEC20F0AA
:101EE00028C001F1019F019D29C000F10101B2EC60
:101EF0001FF02FC182F40401300E82273BEC0BF05F
:101F000030C182F40401300E82273BEC0BF031C16A
:101F100082F40401300E82273BEC0BF032C182F4D4
:101F20000401300E82273BEC0BF033C182F4040134
:101F3000300E82273BEC0BF004012C0E826F3BEC41
:101F40000BF00FEC20F02AC001F12BC000F1D8906B
:101F500001330033D890013300330101B2EC1FF09C
:101F60002FC182F40401300E82273BEC0BF030C10C
:101F700082F40401300E82273BEC0BF031C182F475
:101F80000401300E82273BEC0BF032C182F40401D5
:101F9000300E82273BEC0BF033C182F40401300E8B
:101FA00082273BEC0BF054EF19F0FC0E2FEC09F0FC
:101FB000E8CF0BF003018351520AD8B40CEF10F0B4
:101FC00003018351720AD8B40FEF10F0030183515B
:101FD000500AD8B412EF10F003018351700AD8B43C
:101FE00015EF10F003018351550AD8B418EF10F023
:101FF00003018351750AD8B41BEF10F0030183511C
:10200000430AD8B424EF10F003018351630AD8B413
:1020100027EF10F030EF10F00B902AEF10F00B804C
:102020002AEF10F00B922AEF10F00B822AEF10F03B
:102030000B942AEF10F00B842AEF10F00B962AEF86
:1020400010F00B862AEF10F00B982AEF10F00B8897
:102050002AEF10F0FC0E0C6E0BC00BF018EC09F020
:102060000401590E826F3BEC0BF011901192119408
:102070001198FC0E2FEC09F0E8CF0BF00BA01180AB
:102080000BA211820BA411840BA8118811A050EF90
:1020900010F00401520E826F3BEC0BF055EF10F084
:1020A0000401720E826F3BEC0BF011A85FEF10F091
:1020B0000401430E826F3BEC0BF064EF10F004015F
:1020C000630E826F3BEC0BF011A26EEF10F0040177
:1020D000500E826F3BEC0BF073EF10F00401700EAA
:1020E000826F3BEC0BF011A47DEF10F00401550E54
:1020F000826F3BEC0BF082EF10F00401750E826FE3
:102100003BEC0BF054EF19F004016D0E826F3BECC9
:102110000BF003018351300AD8B4E1EF10F0030152
:102120008351310AD8B4F4EF10F003018351320A1D
:10213000D8B407EF11F056EF19F081B803D02FB4DF
:1021400054EF19F004014D0E826F3BEC0BF050EC94
:1021500020F084C331F185C332F186C333F101012C
:10216000296B5DEC20F0D4EC1FF003018351300AA1
:10217000D8B4C9EF10F003018351310AD8B4D1EFBC
:1021800010F003018351320AD8B4D9EF10F056EFA2
:1021900019F0FD0E0C6E00C10BF018EC09F0E1EF28
:1021A00010F0FE0E0C6E00C10BF018EC09F0F4EF0D
:1021B00010F0FF0E0C6E00C10BF018EC09F007EFE9
:1021C00011F00401300E826F3BEC0BF004012C0E79
:1021D000826F3BEC0BF00FEC20F0FD0E2FEC09F0C2
:1021E000E8CF00F118EF11F00401310E826F3BECE3
:1021F0000BF004012C0E826F3BEC0BF00FEC20F087
:10220000FE0E2FEC09F0E8CF00F118EF11F00401F9
:10221000320E826F3BEC0BF00FEC20F004012C0E21
:10222000826F3BEC0BF0FF0E2FEC09F0E8CF00F1D2
:10223000B2EC1FF031C182F40401300E82273BEC76
:102240000BF032C182F40401300E82273BEC0BF01C
:1022500033C182F40401300E82273BEC0BF054EFC3
:1022600019F081B803D02FB227EF12F083C32AF1FF
:1022700084C32BF185C32CF186C32DF187C32EF1C6
:1022800088C32FF189C330F18AC331F18BC332F196
:102290008CC333F101015DEC20F0D4EC1FF0160E7D
:1022A0000C6E00C10BF018EC09F0170E0C6E01C19A
:1022B0000BF018EC09F0180E0C6E02C10BF018ECC4
:1022C00009F0190E0C6E03C10BF018EC09F000C1F7
:1022D0008AF101C18BF102C18CF103C18DF100C102
:1022E0008EF101C18FF102C190F103C191F127EF8D
:1022F00012F081B803D02FB227EF12F083C32AF176
:1023000084C32BF185C32CF186C32DF187C32EF135
:1023100088C32FF189C330F18AC331F18BC332F105
:102320008CC333F101015DEC20F0D4EC1FF000C14F
:102330008AF101C18BF102C18CF103C18DF100C1A1
:102340008EF101C18FF102C190F103C191F127EF2C
:1023500012F081B803D02FB227EF12F083C32AF115
:1023600084C32BF185C32CF186C32DF187C32EF1D5
:1023700088C32FF189C330F18AC331F18CC332F1A4
:102380008DC333F101015DEC20F0D4EC1FF00101AD
:10239000000E046F000E056F010E066F000E076F32
:1023A00025EC1FF01A0E0C6E00C10BF018EC09F0B2
:1023B0001B0E0C6E01C10BF018EC09F01C0E0C6E1C
:1023C00002C10BF018EC09F01D0E0C6E03C10BF0EE
:1023D00018EC09F000C192F101C193F102C194F12E
:1023E00003C195F127EF12F081B803D02FB227EF88
:1023F00012F083C32AF184C32BF185C32CF186C369
:102400002DF187C32EF188C32FF189C330F18AC320
:1024100031F18CC332F18DC333F101015DEC20F059
:10242000D4EC1FF00101000E046F000E056F010EC9
:10243000066F000E076F25EC1FF000C192F101C17D
:1024400093F102C194F103C195F127EF12F0160E3A
:102450002FEC09F0E8CF00F1170E2FEC09F0E8CFD0
:1024600001F1180E2FEC09F0E8CF02F1190E2FEC54
:1024700009F0E8CF03F1B2EC1FF075EC1DF0040198
:10248000730E826F3BEC0BF004012C0E826F3BEC61
:102490000BF08AC100F18BC101F18CC102F18DC139
:1024A00003F1B2EC1FF075EC1DF00401730E826FA6
:1024B0003BEC0BF004012C0E826F3BEC0BF01A0E80
:1024C0002FEC09F0E8CF00F11B0E2FEC09F0E8CF5C
:1024D00001F11C0E2FEC09F0E8CF02F11D0E2FECDC
:1024E00009F0E8CF03F171EC19F004012C0E826FB2
:1024F0003BEC0BF092C100F193C101F194C102F1E8
:1025000095C103F171EC19F045EC0BF056EF19F0A1
:102510000401690E826F3BEC0BF004012C0E826FFC
:102520003BEC0BF00101040E006F000E016F000E7A
:10253000026F000E036FB2EC1FF02CC182F4040195
:10254000300E82273BEC0BF02DC182F40401300EDB
:1025500082273BEC0BF02EC182F40401300E82275F
:102560003BEC0BF02FC182F40401300E82273BECD0
:102570000BF030C182F40401300E82273BEC0BF0EB
:1025800031C182F40401300E82273BEC0BF032C1E2
:1025900082F40401300E82273BEC0BF033C182F44D
:1025A0000401300E82273BEC0BF004012C0E826FED
:1025B0003BEC0BF00101030E006F000E016F000EEB
:1025C000026F000E036FB2EC1FF02CC182F4040105
:1025D000300E82273BEC0BF02DC182F40401300E4B
:1025E00082273BEC0BF02EC182F40401300E8227CF
:1025F0003BEC0BF02FC182F40401300E82273BEC40
:102600000BF030C182F40401300E82273BEC0BF05A
:1026100031C182F40401300E82273BEC0BF032C151
:1026200082F40401300E82273BEC0BF033C182F4BC
:102630000401300E82273BEC0BF004012C0E826F5C
:102640003BEC0BF00101370E006F000E016F000E26
:10265000026F000E036FB2EC1FF02CC182F4040174
:10266000300E82273BEC0BF02DC182F40401300EBA
:1026700082273BEC0BF02EC182F40401300E82273E
:102680003BEC0BF02FC182F40401300E82273BECAF
:102690000BF030C182F40401300E82273BEC0BF0CA
:1026A00031C182F40401300E82273BEC0BF032C1C1
:1026B00082F40401300E82273BEC0BF033C182F42C
:1026C0000401300E82273BEC0BF004012C0E826FCC
:1026D0003BEC0BF0200EF86EF76AF66A0401090075
:1026E000F5CF82F43BEC0BF00900F5CF82F43BEC24
:1026F0000BF00900F5CF82F43BEC0BF00900F5CFAD
:1027000082F43BEC0BF00900F5CF82F43BEC0BF0CC
:102710000900F5CF82F43BEC0BF00900F5CF82F411
:102720003BEC0BF00900F5CF82F43BEC0BF045ECF1
:102730000BF056EF19F081B803D02FB0EBEF13F088
:102740008351630AD8A454EF19F08451610AD8A4C4
:1027500054EF19F085516C0AD8A454EF19F0865142
:10276000410A42E08651440A1BE08651420AD8B42D
:1027700007EF14F08651350AD8B4E0EF1AF086510D
:10278000360AD8B435EF1BF08651370AD8B49EEF1D
:102790001BF08651380AD8B4FCEF1BF054EF19F047
:1027A0000798079A04017A0E826F3BEC0BF0040144
:1027B000780E826F3BEC0BF00401640E826F3BECF1
:1027C0000BF081A8EBEF13F00401550E826F3BEC88
:1027D0000BF0F0EF13F004014C0E826F3BEC0BF0AA
:1027E00045EC0BF056EF19F00788079A04017A0EB2
:1027F000826F3BEC0BF00401410E826F3BEC0BF05F
:102800000401610E826F3BEC0BF0E1EF13F00798CF
:10281000078A04017A0E826F3BEC0BF00401420E32
:10282000826F3BEC0BF00401610E826F3BEC0BF00E
:10283000E1EF13F00101666725EF14F0676725EFFC
:1028400014F0686725EF14F0696715D04F6730EF13
:1028500014F0506730EF14F0516730EF14F0526706
:102860000AD00101000E006F000E016F000E026F12
:10287000000E036F120011B80AD00101620E046F3E
:10288000010E056F000E066F000E076F09D00101E3
:10289000A70E046F020E056F000E066F000E076F85
:1028A00066C100F167C101F168C102F169C103F1BC
:1028B00014EC1FF003BFCDEF14F0119A119C01012D
:1028C000000E046FA80E056F550E066F020E076FFF
:1028D00066C100F167C101F168C102F169C103F18C
:1028E00066C186F167C187F168C188F169C189F164
:1028F00014EC1FF003BF0BD00101000E866FA80E71
:10290000876F550E886F020E896F118A119C0E0E0B
:102910002FEC09F0E8CF18F10F0E2FEC09F0E8CFFB
:1029200019F1100E2FEC09F0E8CF1AF1110E2FEC6F
:1029300009F0E8CF1BF15DEC1EF086C104F187C100
:1029400005F188C106F189C107F114EC1FF0078277
:1029500021EC1EF05DEC1EF0079221EC1EF086C10A
:1029600000F187C101F188C102F189C103F1079229
:1029700021EC1EF0CC0E046FE00E056F870E066F83
:10298000050E076F14EC1FF000C118F101C119F119
:1029900002C11AF103C11BF13BD0119C119A010134
:1029A000800E006F1A0E016F060E026F000E036F8D
:1029B0004FC104F150C105F151C106F152C107F1F7
:1029C00014EC1FF003AF05D00FEC20F0118C119A1E
:1029D00012000E0E2FEC09F0E8CF18F10F0E2FECBD
:1029E00009F0E8CF19F1100E2FEC09F0E8CF1AF139
:1029F000110E2FEC09F0E8CF1BF14FC100F150C1CF
:102A000001F151C102F152C103F1078221EC1EF024
:102A100018C100F119C101F11AC102F11BC103F182
:102A200012000401730E826F3BEC0BF004012C0EBC
:102A3000826F3BEC0BF0078462C166F163C167F102
:102A400064C168F165C169F14BC14FF14CC150F1EE
:102A50004DC151F14EC152F157C159F158C15AF10E
:102A6000079437EC15F045EC0BF056EF19F066C102
:102A700000F167C101F168C102F169C103F101010F
:102A8000B2EC1FF075EC1DF00401630E826F3BEC9D
:102A90000BF004012C0E826F3BEC0BF04FC100F1E8
:102AA00050C101F151C102F152C103F10101B2EC77
:102AB0001FF075EC1DF00401660E826F3BEC0BF00D
:102AC00004012C0E826F3BEC0BF00FEC20F059C18F
:102AD00000F15AC101F10101B2EC1FF075EC1DF0DB
:102AE0000401740E826F3BEC0BF0120010820401A3
:102AF000530E826F3BEC0BF004012C0E826F3BEC0B
:102B00000BF083C32AF184C32BF185C32CF186C358
:102B10002DF187C32EF188C32FF189C330F18AC309
:102B200031F18BC332F18CC333F101015DEC20F044
:102B3000D4EC1FF000C166F101C167F102C168F178
:102B400003C169F18EC32AF18FC32BF190C32CF11D
:102B500091C32DF192C32EF193C32FF194C330F1A1
:102B600095C331F196C332F197C333F101015DECA6
:102B700020F0D4EC1FF000C14FF101C150F102C1AF
:102B800051F103C152F150EC20F099C32FF19AC3D7
:102B900030F19BC331F19CC332F19DC333F101018C
:102BA0005DEC20F0D4EC1FF000C159F101C15AF1E5
:102BB00037EC15F004012C0E826F3BEC0BF0F1EFBB
:102BC00015F0118E19A002D019AE108C18BE02D0CB
:102BD00018A4108E03018251520A02E10F8201D023
:102BE0000F928251750A02E1108401D01094825133
:102BF000550A02E1108601D0109611A003D011A44D
:102C000001D01084078410B25FEF16F010A44BEFD0
:102C100016F0B6C166F1B7C167F1B8C168F1B9C1C4
:102C200069F1BAC16AF1BBC16BF1BCC16CF1BDC144
:102C30006DF1BEC16EF1BFC16FF1C0C170F1C1C114
:102C400071F1C2C172F1C3C173F1C4C174F1C5C1E4
:102C500075F1C6C176F1C7C177F1C8C178F1C9C1B4
:102C600079F1CAC17AF1CBC17BF1CCC17CF1CDC184
:102C70007DF1CEC17EF1CFC17FF1D0C180F1D1C154
:102C800081F1D2C182F1D3C183F1D4C184F1D5C124
:102C900085F153EF16F062C166F163C167F164C15B
:102CA00068F165C169F14BC14FF14CC150F14DC1A3
:102CB00051F14EC152F157C159F158C15AF107941F
:102CC0000FA081EF16F0010192676EEF16F0936787
:102CD0006EEF16F094676EEF16F0956772EF16F0D0
:102CE00081EF16F01AEC14F092C104F193C105F1D2
:102CF00094C106F195C107F114EC1FF003BF1CEF5E
:102D000019F01AEC14F00101000E046F000E056FAB
:102D1000010E066F000E076F45EC1FF011A02AD0C0
:102D200011A228D0B2EC1FF0296701D005D0040110
:102D30002D0E826F3BEC0BF030C182F40401300E9B
:102D400082273BEC0BF031C182F40401300E822764
:102D50003BEC0BF032C182F40401300E82273BECD5
:102D60000BF033C182F40401300E82273BEC0BF0F0
:102D700045EC0BF012A8C3D012981AC01BF01B3AF6
:102D80001B42070E1B1600011B50000AD8B44DEF62
:102D900017F000011B50010AD8B4D9EF16F000015A
:102DA0001B50020AD8B4D7EF16F07FEF17F07FEF71
:102DB00017F00FEC20F02AC001F12BC000F1D890E1
:102DC00001330033D890013300330101630E046FE7
:102DD000000E056F000E066F000E076F45EC1FF02A
:102DE000280E046F000E056F000E066F000E076FB1
:102DF00014EC1FF000C12DF00FEC20F028C001F101
:102E0000019F019D29C000F10101A40E046F000E75
:102E1000056F000E066F000E076F45EC1FF000C136
:102E20002CF000C104F101C105F102C106F103C19A
:102E300007F1640E006F000E016F000E026F000EAE
:102E4000036F14EC1FF0050E046F000E056F000EEB
:102E5000066F000E076F45EC1FF000C104F101C1C1
:102E600005F102C106F103C107F10FEC20F02DC0FE
:102E700000F114EC1FF000C12EF02EC0E8FF050F8A
:102E80002D5C03E78A847FEF17F02EC0E8FF0A0F5E
:102E90002D5C01E68A947FEF17F000C124F101C197
:102EA00025F102C126F103C127F10FEC20F015EC4A
:102EB00020F01A501F0BE8CF00F10101640E046FDF
:102EC000000E056F000E066F000E076F25EC1FF059
:102ED00024C104F125C105F126C106F127C107F17E
:102EE00014EC1FF003BF02D08A9401D08A8424C15D
:102EF00000F125C101F126C102F127C103F100C192
:102F000024F101C125F102C126F103C127F110AE60
:102F10004DD0109E00C108F101C109F102C10AF1B2
:102F200003C10BF1B2EC1FF030C1D6F131C1D7F1C2
:102F300032C1D8F133C1D9F108C100F109C101F1A1
:102F40000AC102F10BC103F101016C0E046F070EFF
:102F5000056F000E066F000E076F14EC1FF003BF25
:102F600004D00101550EDA6F1CD008C100F109C16F
:102F700001F10AC102F10BC103F10101A40E046FBA
:102F8000060E056F000E066F000E076F14EC1FF0A3
:102F900003BF04D001017F0EDA6F03D00101FF0EE1
:102FA000DA6F1C8E11AE1CEF19F0119E24C100F1D6
:102FB00025C101F126C102F127C103F111A005D0FD
:102FC00011A203D00FB01CEF19F010A4EFEF17F00F
:102FD0000401750E826F3BEC0BF0F4EF17F0040167
:102FE000720E826F3BEC0BF004012C0E826F3BECF7
:102FF0000BF0B2EC1FF0296703EF18F00401200E6C
:10300000826F06EF18F004012D0E826F3BEC0BF07F
:1030100030C182F40401300E82273BEC0BF031C149
:1030200082F40401300E82273BEC0BF004012E0EDB
:10303000826F3BEC0BF032C182F40401300E822728
:103040003BEC0BF033C182F40401300E82273BECE1
:103050000BF004016D0E826F3BEC0BF004012C0EA3
:10306000826F3BEC0BF04FC100F150C101F151C137
:1030700002F152C103F10101B2EC1FF075EC1DF039
:103080000401480E826F3BEC0BF004017A0E826F54
:103090003BEC0BF004012C0E826F3BEC0BF066C195
:1030A00000F167C101F168C102F169C103F10101D9
:1030B000B2EC1FF075EC1DF00401630E826F3BEC67
:1030C0000BF004012C0E826F3BEC0BF066C100F19B
:1030D00067C101F168C102F169C103F101010A0E82
:1030E000046F000E056F000E066F000E076F25ECD3
:1030F0001FF0000E046F120E056F000E066F000E1B
:10310000076F45EC1FF0B2EC1FF02AC182F40401F6
:10311000300E82273BEC0BF02BC182F40401300E01
:1031200082273BEC0BF02CC182F40401300E822785
:103130003BEC0BF02DC182F40401300E82273BECF6
:103140000BF02EC182F40401300E82273BEC0BF011
:103150002FC182F40401300E82273BEC0BF030C10A
:1031600082F40401300E82273BEC0BF004012E0E9A
:10317000826F3BEC0BF031C182F40401300E8227E8
:103180003BEC0BF032C182F40401300E82273BECA1
:103190000BF033C182F40401300E82273BEC0BF0BC
:1031A0000401730E826F3BEC0BF004012C0E826F56
:1031B0003BEC0BF00FEC20F059C100F15AC101F1CA
:1031C00080EC1AF00FB2E8EF18F00FA01AEF19F028
:1031D00004012C0E826F3BEC0BF0200EF86EF76AA8
:1031E000F66A04010900F5CF82F43BEC0BF009000C
:1031F000F5CF82F43BEC0BF00900F5CF82F43BEC09
:103200000BF00900F5CF82F43BEC0BF00900F5CF91
:1032100082F43BEC0BF00900F5CF82F43BEC0BF0B1
:103220000900F5CF82F43BEC0BF00900F5CF82F4F6
:103230003BEC0BF045EC0BF00F9056EF19F004014E
:10324000630E826F3BEC0BF004012C0E826F3BECA3
:103250000BF05CEC19F004012C0E826F3BEC0BF0D0
:10326000CFEC19F004012C0E826F3BEC0BF04BEC11
:103270001AF004012C0E826F3BEC0BF00101F80EEA
:10328000006FCD0E016F660E026F030E036F71ECBF
:1032900019F004012C0E826F3BEC0BF061EC1AF07C
:1032A00045EC0BF056EF19F045EC0BF00301C26B47
:1032B0000790109265EF1CF0D8900E0E2FEC09F0DD
:1032C000E8CF00F10F0E2FEC09F0E8CF01F1100E5E
:1032D0002FEC09F0E8CF02F1110E2FEC09F0E8CF46
:1032E00003F10101000E046F000E056F010E066F61
:1032F000000E076F45EC1FF0B2EC1FF02AC182F4FC
:103300000401300E82273BEC0BF02BC182F4040148
:10331000300E82273BEC0BF02CC182F40401300EFE
:1033200082273BEC0BF02DC182F40401300E822782
:103330003BEC0BF02EC182F40401300E82273BECF3
:103340000BF02FC182F40401300E82273BEC0BF00E
:1033500030C182F40401300E82273BEC0BF031C106
:1033600082F40401300E82273BEC0BF004012E0E98
:10337000826F3BEC0BF032C182F40401300E8227E5
:103380003BEC0BF033C182F40401300E82273BEC9E
:103390000BF004016D0E826F3BEC0BF01200120E6D
:1033A0002FEC09F0E8CF00F1130E2FEC09F0E8CF75
:1033B00001F1140E2FEC09F0E8CF02F1150E2FECFD
:1033C00009F0E8CF03F101010A0E046F000E056F4A
:1033D000000E066F000E076F25EC1FF0000E046F45
:1033E000120E056F000E066F000E076F45EC1FF002
:1033F000B2EC1FF02AC182F40401300E82273BECAC
:103400000BF02BC182F40401300E82273BEC0BF051
:103410002CC182F40401300E82273BEC0BF02DC14D
:1034200082F40401300E82273BEC0BF02EC182F4B3
:103430000401300E82273BEC0BF02FC182F4040113
:10344000300E82273BEC0BF030C182F40401300EC9
:1034500082273BEC0BF004012E0E826F3BEC0BF04D
:1034600031C182F40401300E82273BEC0BF032C1F3
:1034700082F40401300E82273BEC0BF033C182F45E
:103480000401300E82273BEC0BF00401730E826FB7
:103490003BEC0BF012000A0E2FEC09F0E8CF00F124
:1034A0000B0E2FEC09F0E8CF01F10C0E2FEC09F018
:1034B000E8CF02F10D0E2FEC09F0E8CF03F180EF19
:1034C0001AF0060E2FEC09F0E8CF00F1070E2FECF2
:1034D00009F0E8CF01F1080E2FEC09F0E8CF02F176
:1034E000090E2FEC09F0E8CF03F180EF1AF001018B
:1034F0000FEC20F0078457C100F158C101F1079487
:103500000101E80E046F800E056F000E066F000EBD
:10351000076F25EC1FF0000E046F040E056F000E00
:10352000066F000E076F45EC1FF0880E046F130E38
:10353000056F000E066F000E076F14EC1FF00A0EE9
:10354000046F000E056F000E066F000E076F45EC4E
:103550001FF0B2EC1FF001012967B4EF1AF004016B
:10356000200E826FB7EF1AF004012D0E826F3BEC34
:103570000BF030C182F40401300E82273BEC0BF0DB
:1035800031C182F40401300E82273BEC0BF032C1D2
:1035900082F40401300E82273BEC0BF004012E0E66
:1035A000826F3BEC0BF033C182F40401300E8227B2
:1035B0003BEC0BF00401430E826F3BEC0BF012006E
:1035C00087C32AF188C32BF189C32CF18AC32DF15B
:1035D0008BC32EF18CC32FF18DC330F18EC331F12B
:1035E00090C332F191C333F10101296B5DEC20F0FE
:1035F000D4EC1FF00101000E046F000E056F010EE8
:10360000066F000E076F25EC1FF00E0E0C6E00C14A
:103610000BF018EC09F00F0E0C6E01C10BF018EC5A
:1036200009F0100E0C6E02C10BF018EC09F0110E2F
:103630000C6E03C10BF018EC09F004017A0E826FD6
:103640003BEC0BF004012C0E826F3BEC0BF0040101
:10365000350E826F3BEC0BF004012C0E826F3BECBD
:103660000BF05CEC19F0F0EF13F087C32AF188C37C
:103670002BF189C32CF18AC32DF18BC32EF18CC39E
:103680002FF18DC330F18EC331F190C332F191C36C
:1036900033F10101296B5DEC20F0D4EC1FF0880EB2
:1036A000046F130E056F000E066F000E076F19EC06
:1036B0001FF0000E046F040E056F000E066F000E63
:1036C000076F25EC1FF00101E80E046F800E056FF7
:1036D000000E066F000E076F45EC1FF00A0E0C6E11
:1036E00000C10BF018EC09F00B0E0C6E01C10BF0D1
:1036F00018EC09F00C0E0C6E02C10BF018EC09F07E
:103700000D0E0C6E03C10BF018EC09F004017A0EDB
:10371000826F3BEC0BF004012C0E826F3BEC0BF044
:103720000401360E826F3BEC0BF004012C0E826F0D
:103730003BEC0BF04BEC1AF0F0EF13F087C32AF1DF
:1037400088C32BF189C32CF18AC32DF18BC32EF1D1
:103750008CC32FF18DC330F18FC331F190C332F19F
:1037600091C333F101015DEC20F0D4EC1FF0000EA9
:10377000046F120E056F000E066F000E076F25EC2A
:103780001FF001010A0E046F000E056F000E066F98
:10379000000E076F45EC1FF0120E0C6E00C10BF00F
:1037A00018EC09F0130E0C6E01C10BF018EC09F0C7
:1037B000140E0C6E02C10BF018EC09F0150E0C6E15
:1037C00003C10BF018EC09F004017A0E826F3BEC98
:1037D0000BF004012C0E826F3BEC0BF00401370E52
:1037E000826F3BEC0BF004012C0E826F3BEC0BF074
:1037F000CFEC19F0F0EF13F087C32AF188C32BF157
:1038000089C32CF18AC32DF18BC32EF18CC32FF108
:103810008DC330F18EC331F190C332F191C333F1D6
:103820000101296B5DEC20F0D4EC1FF0880E046FD1
:10383000130E056F000E066F000E076F19EC1FF0D8
:10384000000E046F040E056F000E066F000E076F6A
:1038500025EC1FF00101E80E046F800E056F000ECD
:10386000066F000E076F45EC1FF0060E0C6E00C1D0
:103870000BF018EC09F0070E0C6E01C10BF018EC00
:1038800009F0080E0C6E02C10BF018EC09F0090EDD
:103890000C6E03C10BF018EC09F004017A0E826F74
:1038A0003BEC0BF004012C0E826F3BEC0BF004019F
:1038B000380E826F3BEC0BF004012C0E826F3BEC58
:1038C0000BF061EC1AF0F0EF13F081B803D02FB0D9
:1038D00023EF1DF007A8DDEF1CF00101800E006F43
:1038E0001A0E016F060E026F000E036F4BC104F13A
:1038F0004CC105F14DC106F14EC107F114EC1FF0AA
:1039000003BF23EF1DF06FEC1DF04BC100F14CC164
:1039100001F14DC102F14EC103F1078221EC1EF00D
:1039200018C104F119C105F11AC106F11BC107F153
:10393000F80E006FCD0E016F660E026F030E036F5F
:1039400014EC1FF00E0E0C6E00C10BF018EC09F019
:103950000F0E0C6E01C10BF018EC09F0100E0C6E7E
:1039600002C10BF018EC09F0110E0C6E03C10BF044
:1039700018EC09F0078401010FEC20F057C100F1A9
:1039800058C101F107940A0E0C6E00C10BF018EC3F
:1039900009F00B0E0C6E01C10BF018EC09F00C0EC7
:1039A0000C6E02C10BF018EC09F00D0E0C6E03C189
:1039B0000BF018EC09F023EF1DF007AA23EF1DF020
:1039C000078401010FEC20F057C100F158C101F14B
:1039D0000794060E0C6E00C10BF018EC09F0070EF0
:1039E0000C6E01C10BF018EC09F0080E0C6E02C150
:1039F0000BF018EC09F0090E0C6E03C10BF018EC7B
:103A000009F0078462C100F163C101F164C102F1F0
:103A100065C103F10794120E0C6E00C10BF018EC97
:103A200009F0130E0C6E01C10BF018EC09F0140E26
:103A30000C6E02C10BF018EC09F0150E0C6E03C1F0
:103A40000BF018EC09F00798079A040180518119CE
:103A50007F0B0DE09EA8FED714EE00F081517F0B86
:103A6000E126E750812B0F01AD6E25EF1DF092EF9F
:103A70000AF018C100F119C101F11AC102F11BC10C
:103A800003F1000E046F000E056F010E066F000EAD
:103A9000076F45EC1FF029A164EF1DF02051D8B449
:103AA00064EF1DF018C100F119C101F11AC102F152
:103AB0001BC103F1000E046F000E056F0A0E066FA6
:103AC000000E076F45EC1FF01200010104510013B6
:103AD000055101130651021307510313120001018E
:103AE000186B196B1A6B1B6B12002AC182F404014C
:103AF000300E82273BEC0BF02BC182F40401300E18
:103B000082273BEC0BF02CC182F40401300E82279B
:103B10003BEC0BF02DC182F40401300E82273BEC0C
:103B20000BF02EC182F40401300E82273BEC0BF027
:103B30002FC182F40401300E82273BEC0BF030C120
:103B400082F40401300E82273BEC0BF031C182F489
:103B50000401300E82273BEC0BF032C182F40401E9
:103B6000300E82273BEC0BF033C182F40401300E9F
:103B700082273BEC0BF012002FC182F40401300EBF
:103B800082273BEC0BF030C182F40401300E822717
:103B90003BEC0BF031C182F40401300E82273BEC88
:103BA0000BF032C182F40401300E82273BEC0BF0A3
:103BB00033C182F40401300E82273BEC0BF012007B
:103BC000060E1E6E060E1F6E060E206E1E2EE6EFF1
:103BD0001DF01F2EE6EF1DF0202EE6EF1DF08B846A
:103BE000020E1E6E020E1F6E020E206E1E2EF6EFCD
:103BF0001DF01F2EF6EF1DF0202EF6EF1DF08B941A
:103C00001200FF0E1F6E1FC020F0030E1E6E8B846D
:103C10001E2E07EF1EF0030E1E6E202E07EF1EF065
:103C20008B941FC020F0030E1E6E1E2E15EF1EF08B
:103C3000030E1E6E203E15EF1EF01F2E03EF1EF02A
:103C400012000101005305E1015303E1025301E1B8
:103C5000002BE4EC1EF00FEC20F03951006F3A51CC
:103C6000016F420E046F4B0E056F000E066F000EC3
:103C7000076F25EC1FF000C104F101C105F102C17D
:103C800006F103C107F118C100F119C101F11AC110
:103C900002F11BC103F107B252EF1EF019EC1FF045
:103CA00054EF1EF014EC1FF000C118F101C119F11E
:103CB00002C11AF103C11BF112000FEC20F059C12F
:103CC00000F15AC101F1060E2FEC09F0E8CF04F122
:103CD000070E2FEC09F0E8CF05F1080E2FEC09F0E4
:103CE000E8CF06F1090E2FEC09F0E8CF07F114EC4C
:103CF0001FF000C124F101C125F102C126F103C169
:103D000027F1290E046F000E056F000E066F000EDE
:103D1000076F25EC1FF0EE0E046F430E056F000ECB
:103D2000066F000E076F19EC1FF024C104F125C1C6
:103D300005F126C106F127C107F125EC1FF000C1EE
:103D40001CF101C11DF102C11EF103C11FF1120ED0
:103D50002FEC09F0E8CF04F1130E2FEC09F0E8CFB7
:103D600005F1140E2FEC09F0E8CF06F1150E2FEC3B
:103D700009F0E8CF07F10D0E006F000E016F000E85
:103D8000026F000E036F25EC1FF0180E046F000E7B
:103D9000056F000E066F000E076F45EC1FF01CC18B
:103DA00004F11DC105F11EC106F11FC107F119EC97
:103DB0001FF06A0E046F2A0E056F000E066F000ECC
:103DC000076F14EC1FF01200BF0EFA6E200E3A6F50
:103DD000396BD8900037013702370337D8B0F5EF89
:103DE0001EF03A2FEAEF1EF039073A070353D8B412
:103DF00012000331070B80093F6F03390F0B010FCE
:103E0000396F80EC5FF0406F390580EC5FF0405D0A
:103E1000405F396B3F33D8B0392739333FA90AEFB8
:103E20001FF0405139271200010134EC20F0D8B0C6
:103E30001200010103510719346FF7EC1FF0D890FD
:103E40000751031934AF800F12000101346B1BECD2
:103E500020F0D8A031EC20F0D8B0120006EC20F011
:103E60000FEC20F01F0E366F47EC20F00B35D8B06A
:103E7000F7EC1FF0D8A00335D8B01200362F34EF7E
:103E80001FF034B11EEC20F012000101346B04511C
:103E90000511061107110008D8A01BEC20F0D8A0CE
:103EA00031EC20F0D8B01200086B096B0A6B0B6B79
:103EB00047EC20F01F0E366F47EC20F007510B5DEA
:103EC000D8A46FEF1FF006510A5DD8A46FEF1FF062
:103ED0000551095DD8A46FEF1FF00451085DD8A00B
:103EE00082EF1FF00451085F0551D8A0053D095F1E
:103EF0000651D8A0063D0A5F0751D8A0073D0B5FC9
:103F0000D8900081362F5CEF1FF034B11EEC20F00A
:103F1000346B1BEC20F0D8904BEC20F007510B5D7C
:103F2000D8A49FEF1FF006510A5DD8A49FEF1FF0A1
:103F30000551095DD8A49FEF1FF00451085DD8A07A
:103F4000AEEF1FF0003FAEEF1FF0013FAEEF1FF0EE
:103F5000023FAEEF1FF0032BD8B4120034B11EECB9
:103F600020F012000101346B1BEC20F0D8B01200DD
:103F700050EC20F0200E366F003701370237033740
:103F800011EE33F00A0E376FE7360A0EE75CD8B051
:103F9000E76EE552372FC4EF1FF0362FBCEF1FF04E
:103FA00034B12981D890120001010A0E346F200E1D
:103FB000366F11EE29F03451376F0A0ED890E65261
:103FC000D8B0E726E732372FDFEF1FF00333023395
:103FD00001330033362FD9EF1FF0E750FF0FD8A081
:103FE0000335D8B0120029B11EEC20F012000451A4
:103FF00000270551D8B0053D01270651D8B0063D30
:1040000002270751D8B0073D032712000051086F5F
:104010000151096F02510A6F03510B6F1200010128
:10402000006B016B026B036B12000101046B056BEB
:10403000066B076B12000335D8A012000351800BEA
:10404000001F011F021F031F003F2EEF20F0013F42
:104050002EEF20F0023F2EEF20F0032B342B032510
:1040600012000735D8A012000751800B041F051F4E
:10407000061F071F043F44EF20F0053F44EF20F0E8
:10408000063F44EF20F0072B342B072512000037A2
:10409000013702370337083709370A370B37120061
:1040A0000101296B2A6B2B6B2C6B2D6B2E6B2F6BED
:1040B000306B316B326B336B120001012A510F0BE5
:1040C0002A6F2B510F0B2B6F2C510F0B2C6F2D5177
:1040D0000F0B2D6F2E510F0B2E6F2F510F0B2F6FBC
:1040E00030510F0B306F31510F0B316F32510F0BBD
:1040F000326F33510F0B336F120000011650FF0A5D
:1041000001E11200390EC86E800EC76E280EC66E11
:10411000000EC56E1550000AD8B4B8EF20F0155047
:10412000010AD8B4D1EF20F01550020AD8B4EAEF52
:1041300020F01550030AD8B403EF21F01550040AFB
:10414000D8B42BEF21F01550050AD8B444EF21F074
:104150001550060AD8B45DEF21F01550070AD8B4FF
:1041600076EF21F01550080AD8B48FEF21F0120035
:104170001650000AD8B4AEEF21F01650010AD8B498
:10418000B2EF21F01650020AD8B4B6EF21F0165063
:10419000030AD8B4BAEF21F01650040AD8B42DEFB0
:1041A00022F01650000AD8B4C2EF21F01650010ACE
:1041B000D8B4C6EF21F01650020AD8B4CAEF21F0E5
:1041C0001650030AD8B4CEEF21F01650040AD8B422
:1041D0002DEF22F01650000AD8B4D2EF21F016507D
:1041E000010AD8B4D6EF21F01650020AD8B4DAEF9B
:1041F00021F01650030AD8B4DEEF21F01650040A5D
:10420000D8B42DEF22F01650000AD8B4EBEF21F00D
:104210001650010AD8B4EFEF21F01650020AD8B4B4
:10422000F3EF21F01650030AD8B407EF22F016502E
:10423000040AD8B40BEF22F01650050AD8B40FEFD9
:1042400022F01650060AD8B413EF22F01650070ACF
:10425000D8B416EF22F01650000AD8B41AEF22F0A4
:104260001650010AD8B41EEF22F01650020AD8B434
:1042700022EF22F01650030AD8B426EF22F016508F
:10428000040AD8B429EF22F01650000AD8B431EF4E
:1042900022F01650010AD8B435EF22F01650020A67
:1042A000D8B439EF22F01650030AD8B43DEF22F00B
:1042B0001650040AD8B42DEF22F01650000AD8B4D4
:1042C00047EF22F01650010AD8B44BEF22F01650F7
:1042D000020AD8B44FEF22F01650030AD8B453EFB5
:1042E00022F01650040AD8B42DEF22F01650000A1E
:1042F000D8B454EF22F01650010AD8B458EF22F087
:104300001650020AD8B45CEF22F01650030AD8B453
:1043100060EF22F01650040AD8B42DEF22F01650A8
:10432000000AD8B461EF22F01650010AD8B465EF44
:1043300022F01650020AD8B469EF22F01650030A90
:10434000D8B46DEF22F01650040AD8B46EEF22F004
:104350001650050AD8B471EF22F012009E96C5805F
:10436000162A1200E20EC96E162A1200770EC96EC6
:10437000162A1200020EE86E8AB4E88AE8CFC9FF56
:10438000162A12009E96C580162A1200E20EC96EE9
:10439000162A1200790EC96E162A1200000EC96E76
:1043A000162A12009E96C580162A1200E20EC96EC9
:1043B000162A12007A0EC96E162A120018BC03D0F3
:1043C000DAC1E8FF04D01850E844E8441F09E8CFF8
:1043D000C9FF162A12009E96C580162A1200E20E08
:1043E000C96E162A120011BA03D011BC01D003D035
:1043F000050E156E3ED00101D66703EF22F0100EB8
:10440000C96E05EF22F0D6C1C9FF162A1200D7C126
:10441000C9FF162A1200D8C1C9FF162A1200D9C135
:10442000C9FF162A1200C584162A1200FF0E166E46
:104430001D9E12009E96C580162A1200E20EC96EBD
:10444000162A1200760EC96E162A1200C584162A84
:104450001200FF0E166E1D9E1200C584152A166AE4
:1044600012009E96C580162A1200E20EC96E162A08
:1044700012007B0EC96E162A120011AA04D0230E58
:10448000C96E162A12001C0EC96E162A12009E96BC
:10449000C580162A1200E20EC96E162A12007C0E82
:1044A000C96E162A1200E9D79E96C580162A1200F8
:1044B000E20EC96E162A12007D0EC96E162A12006F
:1044C000DCD79E96C580162A1200E20EC96E162A07
:1044D00012007E0EC96E162A1200CFD7C584162A86
:1044E0001200FF0E166E1D9E12001650FF0AD8B461
:1044F00033EF23F0390EC86E800EC76E280EC66EDD
:10450000000EC56E1550000AD8B48EEF22F015507B
:10451000010AD8B4A2EF22F033EF23F01650000ABC
:10452000D8B4E0EF22F01650010AD8B4E4EF22F03C
:104530001650020AD8B4EEEF22F01650030AD8B48F
:10454000F1EF22F01650000AD8B4F7EF22F016501F
:10455000010AD8B4FBEF22F01650020AD8B405EFD6
:1045600023F01650030AD8B408EF23F01650040ABB
:10457000D8B40EEF23F01650050AD8B411EF23F08B
:104580001650060AD8B417EF23F01650070AD8B40D
:104590001AEF23F01650080AD8B420EF23F0165073
:1045A000090AD8B423EF23F016500A0AD8B429EF29
:1045B00023F016500B0AD8B42CEF23F033EF23F07E
:1045C0009E96C58032EF23F017B004D04E0EC96E10
:1045D00032EF23F0500EC96E32EF23F0C58432EF74
:1045E00023F0152AFF0E166E128033EF23F09E96ED
:1045F000C58032EF23F017B004D04F0EC96E32EFF2
:1046000023F0510EC96E32EF23F0C58632EF23F04E
:10461000C9CF24F0C59AC58832EF23F0C58632EFA2
:1046200023F0C9CF25F0C59AC58832EF23F0C5869F
:1046300032EF23F0C9CF26F0C59AC58832EF23F0B8
:10464000C58632EF23F0C9CF27F0C58AC58832EF7F
:1046500023F0C58432EF23F0FF0E166E12861D9CE8
:1046600033EF23F0162A120012B012D012B213D078
:1046700012B414D012A6120007B01200129624C071
:1046800028F025C029F026C02AF027C02BF0120000
:10469000129012821200129212841200000116501F
:0E46A000FF0A04E11294166A75EC22F0120073
:10BF0000E844F926000C160C2B0C3F0C520C640C68
:10BF1000760C860C960CA50CB30CC10CCF0CDC0C6B
:06BF2000E80CF40C000C1B
:00000001FF
